:1014F60020000A3C2E2E2E3E004950436F6E6E652C
:1015060063745245510A004950436F6E6E656374A9
:10151600000A49504E6F41434B210A003E432C5668
:101526002C43432CC0E4E0EFF2E5F020D1E8EDEAED
:10153600EEEC49500A003E432C4D41432C253032F7
:1015460062583A25303262583A25303262583A2586
:10155600303262583A25303262583A253032625873
:101566002C4D414320E0E4F0E5F10A003E432C56C1
:1015760045522C20332E3220EEF22025732025737F
:101586002CC2E5F0F1E8FF20495020ECEEE4F3EB45
:10159600FF0A004A756E203235203230303900316C
:1015A600333A35383A3034003E432C4C442C5052B2
:1015B6004F473A20202020202020202020202020B5
:1015C6002020202020202020202020202020202015
:1015D6002020202020202020202020202020202005
:1015E60020202020202020202020202020202020F5
:1015F60020202020202020202CC4E0F2E020EFF044
:10160600EEF8E8E2EAE828F4E0E9EB290A003E2AE7
:101616002C312CCEF1EDEEE2EDFBE520EFE0F0E033
:10162600ECE5F2F0FB20F1E5F2E5E2EEE3EE20E890
:10163600EDF2E5F0F4E5E9F1E00A003E412C413037
:10164600312C2562752E2562752E2562752E256232
:10165600752C495020E0E4F0E5F120E0E4E0EFF2FB
:10166600E5F0E00A003E412C4130322C2562752E11
:101676002562752E2562752E2562752C495020E04F
:10168600E4F0E5F120EEF1ED2E20F1E5F0E2E5F0F3
:10169600E00A003E412C4130332C2562752E25622E
:1016A600752E2562752E2562752C495020E0E4F0D2
:1016B600E5F120F0E5E72E20F1E5F0E2E5F0E00ABD
:1016C600003E412C4130342C2562752E2562752E44
:1016D6002562752E2562752CCCE0F1EAE020F1E555
:1016E600F2E80A003E412C4130352C2562752E2544
:1016F60062752E2562752E2562752CD8EBFEE70ADB
:10170600003E2A2C312CC4EEEF2E20EFE0F0E0EC68
:10171600E5F2F0FB20F1E5F2E5E2EEE3EE20E8ED9E
:10172600F2E5F0F4E5E9F1E00A003E422C533031EF
:101736002C2562752CC6E4E0F2FC20E7E0EFF0EE23
:10174600F1E020F1EEE5E4E8EDE5EDE8FF20EEF26C
:1017560020F1E5F0E2E5F0E00A003E422C5330329B
:101766002C2562752CCEE1ECE5ED20F120F1E5F0BB
:10177600E2E5F0EEEC20E1E5E720EAE2E8F2E0ED72
:10178600F6E8E90A003E422C5330332C2562752CCC
:10179600CFE5F0E5E7E0EFF3F1EA20EFF0E820EF40
:1017A600EEF2E5F0E520F1E2FFE7E820F120F1E5D1
:1017B600F0E2E5F0EEEC0A003E454E440A000A442B
:1017C600756D705820202020203030203031203098
:1017D6003220303320303420303520303620303738
:1017E600203038203039203041203042203043200C
:1017F6003044203045203046000A3A003A20000A9C
:10180600000A44756D70442020202020303020309E
:1018160031203032203033203034203035203036FD
:1018260020303720303820303920304120304220D7
:101836003043203044203045203046004572722027
:101846006B657900526420656570726F6D0A00528F
:1018560064204D454D0A00526420436F64650A00BA
:10186600577269746520436F64650A004465627542
:10187600674950204F4E0A004465627567495020FB
:101886004F46460A00446562756755736572204F78
:101896006E0A00446562756755736572204F464649
:1018A6000A0044656275674D7367204F6E0A0044EF
:1018B600656275674D7367204F46460A00436F6E33
:1018C600666967206C6F636B210A00577220656535
:1018D60070726F6D0A0020536176652065657072BF
:1018E6006F6D210A00457272204D414321004C6FF5
:1018F60061643E3E002A003C4130313D003C4130AF
:10190600323D003C4130333D003C4130343D003CEB
:101916004130353D003C21003C5330313D003C53C5
:1019260030323D003C5330333D003C5330353D00B2
:061936003C5330363D0079
:064E28000113000111005E
:1052AE00C28E438910E4F58B758DB8D2ABD28E22A7
:03001B0002489FF9
:10489F00C0E0C083C082C0D0C28E758B00758DB84A
:1048AF00201C0675A61E75A6E10511D218E513602A
:1048BF00020513E512D39401400215120516E516F1
:1048CF00540F7048D224E516543F7012D216907BC5
:1048DF000FE0600A04F0E0D394B44002D21C907B46
:1048EF000AE0600204F0907588E0600214F0907B9B
:1048FF0010E0D394014003E014F0301B020514E5DF
:10490F0015D394644004D21C80020515E510D3948E
:10491F000140021510D28ED0D0D082D083D0E03299
:10087900C291C290D2B5C2217D027C007F0712527B
:10088900188F28E528646060097D017F6012517422
:10089900D221E4FDFC7F0B1252188F28E52830E69F
:1008A900097D04E4FF125198D2217D017C007F0764
:1008B9001252188F28E5287008FD7FFF125174D253
:1008C90021302103126000C288C2A8C2AA7589001A
:1008D900124C579077C2E0B4FA06A3E064CE607B6D
:1008E900E4F52874BA2528F582E43477F583E4F031
:1008F9000528E528B443EC9077C274FAF0A374CEC6
:10090900F0A374CCF09077C8740AF0E4A3F0A304C0
:10091900F0A3F09077BE74FFF0A3F0A3F0E4A3F086
:100929009077D9740AF0E4F528E5282401FFE43327
:10093900FE74BA2528F582E43477F583E0FD125177
:10094900500528E528C3944340DFE4F5A775A61EA2
:1009590075A6E1907FF0F0A3F080FE9077CD740347
:10096900F0A374CCF0E49077CCF0124521C2B51213
:100979003BD4C21C125008D221C223C2229079FA58
:100989007408F09077387424F0E4A3F09077C2E00B
:1009990090773AF09077C3E090773BF09077C4E096
:1009A90090773CF09077C5E090773DF09077C6E07E
:1009B90090773EF09077C7E090773FF0751201E4A9
:1009C9009079FBF0C21DC21EC21FC220202118AFA0
:1009D90028FE7D03124365E4FF1247597E147FF612
:1009E900E4FBFDFC124072907B0FE060037401F0A0
:1009F900E4907588F0F5149079F9F0F5151252AE76
:100A090075A70775A61E75A6E1D2AFE4F515907511
:100A190088E07003122965907B10E06401701D90D5
:100A290080007410F09080A874FFF0A3F0A3F0A3E5
:100A3900F0E4907B10F0D221C222C223908008E01A
:100A4900F52830E405D21D7410F0E52830E508D208
:100A59001F9080087420F0E52830E608D21E9080A7
:100A6900087440F0E514C394034019908002E4F03F
:100A7900908001F0908000F0E51494064006E4F5BA
:100A8900141250089080A0E07003124D4F9080B866
:100A9900E07003124CD59080D0E07003124FAC90F7
:100AA9008000E07013301D101241799077B5EFF096
:100AB900D394004003120036908002E070069080C3
:100AC90000E06005D21B020A14C21BE4F5149075FC
:100AD90088E06003020A142021129079FCE0600C7E
:100AE9007E147FF812427DE49079FCF0301F1212D7
:100AF90038F29077B5EFF0D394004005E0FF12008B
:100B090021201E03020C8A1234689077B5EFF07029
:100B190003020A149077F9E054BF247F7003020B93
:100B2900F3147003020BCB24026003020C2C202166
:100B3900077E147FFF12427D202503020C8A9077DD
:100B4900D1E070069077D5E06067907B06E0FF9072
:100B590077D1E0B50724907B07E0FE9077D2E0B526
:100B69000618907B08E0FE9077D3E0B5060C907BE1
:100B790009E0FE9077D4E06E60379077D5E06F603A
:100B890003020C8A907B07E0FF9077D6E06F600341
:100B9900020C8A907B08E0FF9077D7E06F60030230
:100BA9000C8A907B09E0FF9077D8E06F6003020C14
:100BB9008AC2199079FB7401F012001E75120102A4
:100BC9000C8A907B0FE060037401F0907AFEE0FFDD
:100BD9009077FBE06F6003020C8A907AFEE004F0E4
:100BE900E4F5129079F9F0020C8A301903020C8AA3
:100BF9009077C8E07003020A149077D9740AF0124A
:100C09005235D219E4F5129079F9F0907B0A04F083
:100C1900E4907AFDF0A3F02021677E157F0D124242
:100C29007D805E907B0FE060037401F03019529073
:100C390077F9E020E74B9077FBE0FF907AFDE0FE43
:100C49006F600D907B05E07007EE146F70338013B1
:100C5900907AFDE004F09077B5E0FFD39404400367
:100C69001251BC9074847482F0A37401F09077FBE4
:100C7900E0907486F07E747F847D03124A42020AF2
:100C890014201903020DA2E5127068121CE8EF6026
:100C9900237E787FF99078FAE02404FD124A429085
:100CA9007B05E070099077D9E0F512020A14E4F5A2
:100CB90012020A14907B0AE0D3943C4036907B05DB
:100CC900E07030907B0A04F01246A4E49078F9F0C1
:100CD900A37412F0907AFEE09078FBF0A374FDF013
:100CE90090758963A2019078FD63A2017F12123188
:100CF900B6809E1200268F28E528B40115907484C9
:100D09007483F0E4A3F07E747F847D02124A420268
:100D19000A14E528D39401401C9074847483F0A3C9
:100D29007401F0E52824FEA3F07E747F847D03120C
:100D39004A42020A14E51264016003020A14907916
:100D4900F9E004F02021077E157F1712427D907784
:100D5900D9E0C394C85004E02432F09079F9E0C393
:100D69009405400DC219E49079FBF012001E020AA5
:100D7900147C7B7D069077CDE0FAA3E0FB7F02121D
:100D89004BD37E787FF99078FAE02404FD124A4229
:100D99009077D9E0F512020A14E5126401600302A2
:100DA9000A149079FBE014604624FE604214700333
:100DB900020E9524046003020A14E4F51420251395
:100DC9009079FB7404F09079F9E05401F0751201FF
:100DD900020A149080027410F0E49079FBF0907983
:100DE900F904F07512FA907B0674FFF0020A149068
:100DF9007B06E07003020E7F9078F97480F090789A
:100E0900FB7401F0E4A3F0A304F0A37430F0A3741D
:100E19007BF0E4F52874002528F582E43479F5831C
:100E2900747DF074012528F582E43479F583E4F0C2
:100E3900E52824079078FAF07C7B7D069077CDE051
:100E4900FAA3E0FB7F02124BD37E787FF9E52824D1
:100E590009FD124A42907B05E0601B125235D219F6
:100E6900E4F5129079F9F0907B0A04F0E4907AFDA8
:100E7900F0A3F0020A14302507E49079FBF080060C
:100E89009079FB7404F07512FA020A1490800274C6
:100E990010F07512059079F9E06401FFF09079FB83
:100EA9007401F0EF70199077D5E06013FCA3E0FDB1
:100EB900A3E0FEA3E0FF907B061224EE020A149041
:100EC90077D1E0FCA3E0FDA3E0FEA3E0FF907B0661
:080ED9001224EE020A1480FE4F
:010EE10022EE
:100036009077FAE0B444047F0180027F009077F95C
:10004600E0B447047E0180027E00EE5F604A90774E
:10005600C2E09077FBF09077C3E09077FCF0907762
:10006600C4E09077FDF09077C5E09077FEF090774A
:10007600C6E09077FFF09077C7E0907800F0907731
:10008600FA7452F090773263A2019080A863A201BD
:100096007F061231B602086F9077B5E0C394085018
:1000A600030208789077C2E0FF9077FBE06F600369
:1000B6000208789077C3E0FF9077FCE06F60030258
:1000C60008789077C4E0FF9077FDE06F6003020840
:1000D600789077C5E0FF9077FEE06F6003020878BE
:1000E6009077C6E0FF9077FFE06F60030208789094
:1000F60077C7E0FF907800E06F600302087890779A
:10010600FAE06444701A9080A8E0B4FF1390773246
:1001160063A2019080A863A2017F061231B6801007
:10012600907736E09080ACF0907737E09080ADF035
:10013600907B0FE060037401F0907B107464F09084
:1001460077FA7452F09077F9E0646D6003020279F1
:100156007BFF7A1579221220E37BFF7A15793C9092
:1001660077C2E0F531A3E0F532A3E0F533A3E0F57D
:1001760034A3E0F535A3E0F5361220E37531FF75BB
:1001860032157533997534FF7535157536A57BFFB0
:100196007A1579721220E37BFF7A1579AE1220E385
:1001A6007BFF7A1679141220E37BFF7A1679419049
:1001B60077C8E0F531A3E0F532A3E0F533A3E0F527
:1001C600341220E37BFF7A16796B9077D1E0F53114
:1001D600A3E0F532A3E0F533A3E0F5341220E37B88
:1001E600FF7A1679999077D5E0F531A3E0F532A339
:1001F600E0F533A3E0F5341220E37BFF7A1679C7E6
:100206009077BEE0F531A3E0F532A3E0F533A3E045
:10021600F5341220E37BFF7A1679EA9077BAE0F597
:1002260031A3E0F532A3E0F533A3E0F5341220E381
:100236007BFF7A1779071220E37BFF7A177930A2C2
:1002460025E433F5311220E37BFF7A177960907B42
:1002560005E0F5311220E37BFF7A17798B907B0F4F
:10026600E0F5311220E3123A637BFF7A1779BE126A
:1002760020E3229077F9E0644C70737E177FC4FB0D
:10028600FDFC124072907801E0F529A3E0F52AE41E
:10029600F52CE529907803F0A3E52AF07E177FFF79
:1002A6007C787D037B02124072E4F52B852A8285D9
:1002B6002983E0FF7403252BF582E43478F583EF78
:1002C600F0052AE52A70020529052BE52BB410DC7A
:1002D6007E187F027C787D037B10124072052CE528
:1002E6002CC3941040AC7E187F0512427D22907775
:1002F600F9E0646C7060F52D7E187F07FBFDFC123B
:100306004072E4F52CE4907803F0A3E52DF07E1717
:100316007FFF7C787D037B02124072E4F52BA82DCB
:10032600E6FF7403252BF582E43478F583EFF005B8
:100336002D052BE52BB410E67E187F027C787D0315
:100346007B10124072052CE52CC3940840B77E182A
:100356007F0512427D229077F9E0644B7061F52BA0
:1003660074EB252BF582E43477F583E0603274EB89
:10037600252BF582E43477F583E0F4602374EB25CE
:100386002BF582E43477F583E0FF7401252BF582A3
:10039600E43478F583E0B50710052BE52BB408C0E7
:1003A6009075887432F002086F9077F97421F030F6
:1003B600210302086F7E187F4212427D02086F9069
:1003C60077F9E0B4521A2021077E187F4A12427D3F
:1003D6009077F97472F07E777FF97D081249BB2217
:1003E6009077F9E0644970452021077E187F551201
:1003F600427D907801E0F529A3E0F52AE4F52B8506
:100406002A82852983E0FF7403252BF582E434785C
:10041600F583EFF0052AE52A70020529052BE52B61
:10042600B480DC7E777FF97D8A1249BB229077F90A
:10043600E0644370462021077E187F5D12427D905E
:100446007801E0F529A3E0F52AE4F52B852A8285D3
:100456002983E493FF7403252BF582E43478F5832E
:10046600EFF0052AE52A70020529052BE52BB48055
:10047600DB7E777FF97D8A1249BB229077F9E064AB
:100486005A70532021077E187F6612427D907801AC
:10049600E0F529A3E0F52A7C787D037B80AF2AAEC0
:1004A6002912511CE4F52B852A82852983E493FFC2
:1004B6007403252BF582E43478F583EFF0052AE5FD
:1004C6002A70020529052BE52BB480DB7E777FF9A0
:1004D6007D8A1249BB229077F9E0644460030205E5
:1004E6006D907801E0FF6444700302086FEFB43149
:1004F6000CC2217E187F7212427D02086F9078012D
:10050600E0B4300CD2217E187F7E12427D02086F45
:10051600907801E0B4320CD2227E187F8B12427D95
:1005260002086F907801E0B4330CC2227E187F99DE
:1005360012427D02086F907801E0B4340CD2237E1B
:10054600187FA812427D02086F907801E0B4350C3E
:10055600C2237E187FB512427D02086F907801E0B3
:10056600FF12528602086F907588E07013202107EB
:100576007E187FC312427D9077F97421F002086FCE
:100586009075887432F09077F9E0FFB45104C2AFE9
:1005960080FEEF645770452021077E187FD11242F6
:1005A6007D907802E09077B5F0E4F52B9077B5E092
:1005B600FFE52BC39F400302086F7403252BF582CA
:1005C600E43478F583E0FF907801E0252B2431F5BB
:1005D60082E43476F583EFF0052B80D09077F9E04E
:1005E600645360030206902021077E187FDC1242C6
:1005F6007D9077C2E0FF90763AE06F703C9077C3CB
:10060600E0FF90763BE06F70309077C4E0FF907625
:100616003CE0B507249077C5E0FF90763DE0B5074E
:10062600189077C6E0FF90763EE0B5070C9077C746
:10063600E0FF90763FE06F60169077F97421F03016
:10064600210302086F7E187FEB12427D02086FE4D9
:10065600F52BE4F515AF2BFE7431252BF582E4342A
:1006660076F583E0FD125150052BE52BC394FE4031
:10067600E1C2AFE4907FF0F0A3F0907FFD74AAF0A2
:10068600A374FFF0A37455F080FE9077F9E0644FF1
:10069600704C907801E0F529A3E0F52AE52A452972
:1006A600700A2021077E187FF412427D2021077EE2
:1006B600187FFB12427DE4F52B7403252BF582E4AB
:1006C6003478F583E0852A82852983F0052AE52A90
:1006D60070020529052BE52BB480DE02086F9077A2
:1006E600F9E0FFB44521907801E0FDA3E0907FF0AA
:1006F600CDF0A3EDF0C2AF907FFD74AAF0A374FF16
:10070600F0A37455F080FEEF6465600302087890EC
:100716007801E0FFA3E0907FF0CFF0A3EFF0E4F5DF
:1007260029F52AD3907FF1E0952A907FF0E095296C
:100736004020E4F515252AFFE5293401FE852A82A5
:10074600852983E0FD125150052AE52A7002052904
:1007560080D17E187FFD124AC9EF4E602012000339
:100766009077C8EFF01200039077C9EFF0120003FC
:100776009077CAEFF01200039077CBEFF07E197FE7
:1007860003124AC9EF4E60201200039077D1EFF0B2
:100796001200039077D2EFF01200039077D3EFF0B8
:1007A6001200039077D4EFF07E197F09124AC9EF41
:1007B6004E60201200039077D5EFF0120003907779
:1007C600D6EFF01200039077D7EFF0120003907780
:1007D600D8EFF07E197F0F124AC9EF4E6020120043
:1007E600039077BEEFF01200039077BFEFF0120090
:1007F600039077C0EFF01200039077C1EFF07E19F7
:100806007F15124AC9EF4E60201200039077BAEFA7
:10081600F01200039077BBEFF01200039077BCEF65
:10082600F01200039077BDEFF0E4F52BE4F515E543
:100836002B2401FFE433FE74BA252BF582E43477CA
:10084600F583E0FD125150052BE52BC3944340DCA4
:10085600C2AFE4907FF0F0A3F0907FFD74AAF0A3FE
:1008660074FFF0A37455F080FE7E777FF97D081241
:0208760049BB7C
:01087800225D
:1050E400AE07EEC39430400BEED394395005EE2452
:1050F400D0FF22EEC39461400BEED394665005EECC
:1051040024A9FF22EEC39441400BEED394465005EC
:08511400EE24C9FF22AF0622C0
:10526C00907731E004F07006907730E004F090779E
:0A527C0030E0FEA3E0FF1251FB2218
:1000030012526C1250E4EFC454F0FEC00612526C4C
:080013001250E4D0E02FFF229F
:104F4F00E4907D04F012526C907D05EFF0C3943025
:104F5F004018E0FFD394395011907D04E02489F577
:104F6F0082E43475F583EFF08011907D04E024899D
:104F7F00F582E43475F583E4F0800C907D04E00451
:104F8F00F0E0D3940840BE753100753200753300E0
:0C4F9F00E4F5347B017A7579891232C484
:014FAB0022E3
:044AC9008E2E8F2F6F
:104ACD00907730E4F0A374FFF012526CEF606EF447
:104ADD00606B852F82852E83E493B507EC753001CD
:104AED00E52F2530F582E4352EF583E4936025908E
:104AFD007731E02530FF907730E03400FE1251FB26
:104B0D00E52F2530F582E4352EF583E493B50704C2
:104B1D00053080CCE52F2530F582E4352EF583E484
:104B2D009370A6E53024FFFFE434FFFE907731E06B
:104B3D002FF0907730E03EF07E007F0122E4FEFF03
:014B4D002245
:104521007E197F1B124AC9EF4E70037F01227E194B
:104531007F1E124AC9EF4E600C12526CEF24D02438
:10454100FF92258002D2257E197F24124AC9EF4E9F
:10455100600C12526CEF24D0907B05F08005E49042
:104561007B05F07E197F2A124AC9EF4E600C125268
:104571006CEF24D0907B0FF08005E4907B0FF07EF0
:10458100197F30124AC9EF4E600C12526CEF24D0E1
:1045910024FF92178002C2179077C263A201907A1A
:1045A100FF63A2017F061231B630173B7E197F36B9
:1045B100124AC9EF4E6030120003907AFFEFF012F9
:1045C1000003907B00EFF0120003907B01EFF012EB
:1045D1000003907B02EFF0120003907B03EFF012D7
:0A45E1000003907B04EFF07F00223E
:105062009079FAE0C3947C40027F0A9079FAE0FEDC
:1050720004F074382EF582E43477F583EFF0BF0A3A
:10508200279079FAE0FF04F074382FF582E4347740
:10509200F583E4F09079FAE0FF124B4E9079FA74BE
:0950A20008F0907739E004F022D7
:10528600BF360BD20EE4F547F548F563F564BF3734
:0452960002C20E2220
:104EF100C2A9438902907CEFE0FFF58C8F8A75D9B6
:104F01000475DA4875DB3175DC4975DD4975DE31CB
:104F1100E4F5E9F5F9F5EBF5FB907CEDE06016754C
:104F2100EC1075ED10E4F5FCF5FD755F08755D108D
:104F3100755E01801375EC8075ED80E4F5FCF5FD7F
:0E4F4100755F80F55D755E10E4F5EEF5FE22FD
:1050AB00E4FEAF8CEFFD907CEEE07003A3E06D604F
:1050BB0005124EF17E01E5D920E2057E02124EF17A
:1050CB00E58920E105124EF17E03D28C75D840752F
:0850DB00B740D2AED2AFAF0620
:0150E30022AA
:030033000237741D
:0B377400C0E0C083C082C0D075D00848
:10377F00C2AF30DC56C3E5EC95EEC3955F5012E552
:10378F005E25ECF5EC30D70405FC801685FCFC803B
:10379F0011C3E5EC955EF5EC30D70415FC8003857D
:1037AF00FCFC300E24854882854783E590F0054860
:1037BF00E54870020547F582854783E5EEF0054839
:1037CF00E5487002054753470FC2DC30D929300E48
:1037DF0024854882854783E590F00548E5487002C7
:1037EF000547F582854783E5EBF00548E54870020C
:1037FF00054753470FC2D930DA6AE55D700405FCFF
:10380F008010E55D25ECF5EC30D70405FC800385D1
:10381F00FCFC300F4DE5495480F527E54925E0F5CF
:10382F00493097020549200D03634901303419E5EA
:10383F004965656006E54965627027755B007560CF
:10384F000085494BC234801A0560E5605407701239
:10385F0053603FE560131313541F244BF8A64975AB
:10386F004900C2DA30DB71E55D700405FD8010E5BB
:10387F005D25EDF5ED30D70405FD800385FDFDE5F4
:10388F0061655C6029E55C54077013E55C131313E5
:10389F00541F2453F8E6F54A200C03634AFFE54A08
:1038AF00339296E54A25E0F54A055C535C3FB292A8
:1038BF00300E23854882854783E590F00548E5481B
:1038CF0070020547F582854783E4F00548E54870A7
:0A38DF0002054753470FC2DBD2AFCA
:0938E900D0D0D082D083D0E032AF
:105008009080007480F09077BA63A201F583F582EE
:1050180063A2017F081231B69077C263A201908023
:105028008863A2017F0A1231B69080927407F0A3B8
:1050380074D0F0A37406F09077CCE0FF9080B1F0C4
:105048009080E1EFF09080957455F0A3F090800087
:0A5058007401F090800974F0F0225A
:104D4F00908009E04410F09080A0E070609080A106
:104D5F007482F09080A874FFF0A3F0A3F0A3F07F0B
:104D6F00039080AEEFF0A374CBF09080007402F04C
:104D7F00907CF41224FA00000000907CF4E0908004
:104D8F0040F0907CF5E0908041F0907CF6E09080D0
:104D9F0042F0907CF7E0908043F0A3E4F0A3F0A3FF
:0D4DAF00F0A3F0908018F0A3F0A3F0A3F0A3
:014DBC0022D4
:104FAC00908009E04440F09080D17482F07F0390AF
:104FBC0080DEEFF0A374CCF09080027402F0907C51
:104FCC00F81224FA00000000907CF8E0908058F071
:104FDC00907CF9E0908059F0907CFAE090805AF047
:104FEC00907CFBE090805BF0A3E4F0A3F0A3F0A333
:0B4FFC00F0908030F0A3F0A3F0A3F0D1
:015007002286
:104CD500908009E04420F09080B8E0706C9080B935
:104CE5007482F07F039080C6EFF07FCDA3EFF07F55
:104CF500039080C4EFF0A374CDF09080C074FFF0F2
:104D0500A3F0A3F0A3F09080017402F0907CFC1254
:104D150024FA00000000907CFCE090804CF0907C30
:104D2500FDE090804DF0907CFEE090804EF0907C10
:104D3500FFE090804FF0A3E4F0A3F0A3F0A3F09080
:094D45008024F0A3F0A3F0A3F018
:014D4E002242
:104BD3008C298D2AA907EAFDE975F018A424ACFFF6
:104BE300E5F034808F82F583EDF0EBFDE975F01885
:104BF300A4FFAEF024ACFBEE34808B82F583A3EDEF
:104C0300F0852A828C83E0FDEF24A8FFEE3480FE3A
:104C13008F82F583EDF0852A828C83A3E08F828EC9
:104C230083A3F0852A82852983A3A3E0FDE975F098
:104C330018A424A8FFE5F03480FE8F82F583A3A394
:104C4300EDF0852A828C83A3A3A3E08F828E83A3B6
:044C5300A3A3F02205
:0649BB008D2EAB07AA06D9
:1049C100908000E030E5079079FC7401F022907C42
:1049D100F4E0FCA3E0FDA3E0FEA3E0F5328E318D0F
:1049E100308C2FAE02AF038E838F8263A201E5313B
:1049F100540744C0F58385328263A201AF2E12327F
:104A010028E4FCFDFEE532252EF532EE3531F53197
:104A1100ED3530F530EC352FF52F908040E52FF056
:104A2100A3E530F0A3E531F0A3E532F09080007406
:104A310020F0AF32AE31AD30AC2F907CF41224EEC9
:014A41002252
:064A42008D29AB07AA0656
:104A4800908002E030E5079079FC7403F022907CB6
:104A5800F8E0FCA3E0FDA3E0FEA3E0F52D8E2C8D8D
:104A68002B8C2AAE02AF038E838F8263A201E52CC2
:104A7800540744D0F583852D8263A201AF291232F1
:104A880028E4FCFDFEE52D2529F52DEE352CF52C29
:104A9800ED352BF52BEC352AF52A908058E52AF0D0
:104AA800A3E52BF0A3E52CF0A3E52DF0908002748C
:104AB80020F0AF2DAE2CAD2BAC2A907CF81224EE52
:014AC80022CB
:024759008F29A6
:10475B00908001E030E5099079FC7402F07F002233
:10476B00907CFCE0FCA3E0FDA3E0FEA3E0F52D8E26
:10477B002C8D2B8C2A907AFF63A201E52C540744D5
:10478B00C8F583852D8263A2017F0612323EE52D8B
:10479B002406F52DE4352CF52CE4352BF52BE435DF
:1047AB002AF52A9079FD63A201E52C540744C8F53C
:1047BB0083852D8263A201AF2912323EE4FCFDFEFC
:1047CB00E52D2529F52DEE352CF52CED352BF52B7F
:1047DB00EC352AF52A90804CE52AF0A3E52BF0A3C3
:1047EB00E52CF0A3E52DF09080017420F0AF2DAEF9
:0D47FB002CAD2BAC2A907CFC1224EEAF29D3
:01480800228D
:104179009081E0E0F5290529052905290529052961
:1041890005290529052905290529908010E0F52C1F
:10419900A3E0F52DA3E0F52EA3E0F52F9081E1E052
:1041A900F5290529052905290529052905290529A6
:1041B900052905290529908014E0F530A3E0F5319A
:1041C900A3E0F532A3E0F533E532B52E08E533B5C2
:1041D9002F037F0022E4F529E532540744E0F583F3
:1041E90085338263A2019077F963A2017F081232B5
:1041F9006E9077FB63A20190773263A2017F06126A
:1042090031B69077F9E0F52AA3E0F52BE4F529908A
:1042190077F9E0702AA3E024F8F529E53254074438
:10422900E0F58385338274082582F582E43583F5C8
:104239008363A2019077F963A201AF2912326EAEAE
:104249002AE4FCFDE533252BF533E5323EF532ED65
:104259003531F531EC3530F530908014E530F0A387
:10426900E531F0A3E532F0A3E533F0908000744026
:03427900F0AF297A
:01427C00221F
:103468009081E6E0F5290529052905290529052979
:1034780005290529052905290529908028E0F52C25
:10348800A3E0F52DA3E0F52EA3E0F52F9081E7E06A
:10349800F5290529052905290529052905290529C4
:1034A80005290529052990802CE0F530A3E0F531A0
:1034B800A3E0F532A3E0F533E4F529E532B52E0AA9
:1034C800E533B52F05C21E0235D4E532540744F062
:1034D800F58385338263A2019077F963A2017F089F
:1034E80012326E9077F9E0F52AA3E0F52BE52B452B
:1034F8002A70099080027410F07F0022907B06E009
:10350800FFF460309077FBE06F600302359B907B9F
:1035180007E0FF9077FCE06F7079907B08E0FF9000
:1035280077FDE06F706D907B09E0FF9077FEE06FAC
:103538006031805F9077FBE0907B06F09077FCE04D
:10354800907B07F09077FDE0907B08F09077FEE0A5
:10355800907B09F09077FFE0FFA3E09077CDCFF064
:10356800A3EFF09077F9E0702AA3E024F8F529E5B5
:1035780032540744F0F58385338274082582F58236
:10358800E43583F58363A2019077F963A201AF293B
:1035980012326EAE2AE4FCFDE533252BF533E53215
:1035A8003EF532ED3531F531EC3530F530AF2FAE33
:1035B8002EAD2DAC2CAB33AA32A931A830D31224AE
:1035C800DD40099080027410F07F002290802CE585
:1035D80030F0A3E531F0A3E532F0A3E533F09080B5
:0635E800027440F0AF295F
:0135EE0022BA
:1038F2009081E3E0F52905290529052905290529EE
:103902000529052905290529052990801CE0F52CA2
:10391200A3E0F52DA3E0F52EA3E0F52F9081E4E0DE
:10392200F529052905290529052905290529052935
:10393200052905290529908020E0F530A3E0F5311D
:10394200A3E0F532A3E0F533E4F529E532B52E0A1A
:10395200E533B52F05C21F023A48E532540744E861
:10396200F58385338263A20190748863A2017F0E7E
:10397200123284907488E0F52AA3E0F52B907490BB
:10398200E0FFF4604A907AFFE0FEEF6E7079A3E008
:10399200FF907491E06F706F907B01E0FF907492E2
:1039A200E06F7063907B02E0FF907493E06F70575A
:1039B200907B03E0FF907494E06F704B907B04E087
:1039C200FF907495E06F703FE4907497F0800890D8
:1039D200749774FFF0D2D9907488E0702AA3E0241F
:1039E200F2F529E532540744E8F583853382740EF3
:1039F2002582F582E43583F58363A201907488639E
:103A0200A201AF29123284AE2AE4FCFDE533252B54
:103A1200F533E5323EF532ED3531F531EC3530F541
:103A220030AF2FAE2EAD2DAC2CAB33AA32A931A8BC
:103A320030D31224DD5006E52B452A70099080010F
:103A42007410F07F0022908020E530F0A3E531F081
:103A5200A3E532F0A3E533F09080017440F0AF2982
:013A62002241
:04427D008E2E8F2FC3
:10428100908000E030E5079079FC7401F022907C89
:10429100F4E0FCA3E0FDA3E0FEA3E0F5358E348D50
:1042A100338C32E535FFE5345407FEE42FF531EE6A
:1042B10034C0F530853182F5837423F00531E53161
:1042C100700205305330C7F582853083740AF005DA
:1042D10031E531700205305330C79077C263A201D6
:1042E10085308385318263A2017F061232287406EC
:1042F1002531F531E43530F530852E83852F826304
:10430100A20185308385318263A20112320CE4FC63
:10431100FDFE907CF4E0F8A3E0F9A3E0FAA3E02F1E
:10432100FFEE3AFEED39FDEC38FCEF2408FFE43EE8
:10433100FEE43DFDE43CFC907CF41224EE907CF420
:10434100E0908040F0907CF5E0908041F0907CF628
:10435100E0908042F0907CF7E0908043F090800004
:034361007420F0D5
:014364002236
:0A4072008E2E8F2F8C308D318B3293
:10407C00908000E030E5079079FC7401F022907C90
:10408C00F4E0FCA3E0FDA3E0FEA3E0F5388E378D51
:10409C00368C35E538FFE5375407FEE42FF534EE62
:1040AC0034C0F533853482F5837423F00534E5345C
:1040BC00700205335333C7F582853383740AF005D8
:1040CC0034E534700205335333C79077C263A201D1
:1040DC0085338385348263A2017F061232287406ED
:1040EC002534F534E43533F533852E83852F8263FF
:1040FC00A20185338385348263A20112320C8F397D
:10410C00EF2534F534E43533F533E532601785307B
:10411C008385318263A20185338385348263A20156
:10412C00AF32123228E53924082532F532FFE4FC8F
:10413C00FDFEE5382FF538EE3537F537ED3536F52C
:10414C0036EC3535F535908040E535F0A3E536F0A5
:10415C00A3E537F0A3E538F09080007420F0AF3879
:0C416C00AE37AD36AC35907CF41224EE7A
:014178002224
:064446008E668F678D6891
:10444C00908000E030E5079079FC7401F022907CBC
:10445C00F4E0FCA3E0FDA3E0FEA3E0F56E8E6D8D11
:10446C006C8C6BE56EFFE56D5407FEE42FF56AEE80
:10447C0034C0F569856A82F5837423F0056AE56AB0
:10448C00700205695369C7F582856983EBF0056A8B
:10449C00E56A700205695369C79077C263A201850A
:1044AC006983856A8263A2017F061232287406250D
:1044BC006AF56AE43569F56985668385678263A266
:1044CC0001856983856A8263A201AF681232287400
:1044DC00082568F568FFE4FCFDFEE56E2FF56EEE31
:1044EC00356DF56DED356CF56CEC356BF56B9080D1
:1044FC0040E56BF0A3E56CF0A3E56DF0A3E56EF081
:10450C009080007420F0AF6EAE6DAD6CAC6B907C97
:04451C00F41224EE83
:014520002278
:024B4E008F4294
:104B5000908000E030E5079079FC7401F022907CB1
:104B6000F4E0FCA3E0FDA3E0FEA3E0F5468E458D56
:104B7000448C43E546FFE5455407FEE42FFFEE3441
:104B8000C090773863A201F5838F8263A201AF42A0
:104B9000123228E4FCFDFEE5462542F546EE354599
:104BA000F545ED3544F544EC3543F543908040E55B
:104BB00043F0A3E544F0A3E545F0A3E546F090807B
:104BC000007420F0AF46AE45AD44AC43907CF41287
:024BD00024EED1
:014BD20022C0
:064365008E298F2AAB0532
:10436B00908000E030E5079079FC7401F022907C9E
:10437B00F4E0FCA3E0FDA3E0FEA3E0F5308E2F8D6F
:10438B002E8C2DE530FFE52F5407FEE42FF52CEE98
:10439B0034C0F52B852C82F5837423F0052CE52C8A
:1043AB007002052B532BC7F582852B83EBF0052C65
:1043BB00E52C7002052B9077C263A201852B8385B8
:1043CB002C8263A2017F061232287406252CF52C51
:1043DB00E4352BF52B532BC7E529852C82852B83B5
:1043EB00F0052CE52C7002052B532BC7F582852B82
:1043FB0083E52AF0052CE52C7002052B532BC7E522
:10440B0030240AF530E4352FF52FE4352EF52EE464
:10441B00352DF52D908040E52DF0A3E52EF0A3E58D
:10442B002FF0A3E530F09080007420F0AF30AE2F6A
:0A443B00AD2EAC2D907CF41224EE9F
:014445002254
:102E8800CEF820E4EBE8EDFB210A000A4173796EE5
:102E9800634F55543A200020000A435243204552BC
:102EA800523A20000A4173796E63494E3A000AD2B9
:102EB800D320EEE4EDEEF1F2E0E4E8E9EDEEE50A28
:102EC80000D2D320330A00C0F0F5D2D10A003F3F28
:102ED8003F0A000089129B24AD36BF48C15AD36C03
:102EE800E57EF78108931AA52CB73EC940DB52ED61
:102EF80064FF76028B109926AF34BD4AC358D16E51
:102F0800E77CF5830A9118A72EB53CCB42D950EF40
:102F180066FD74048D169F20A932BB4CC55ED76828
:102F2800E17AF3850C971EA128B33ACD44DF56E920
:102F380060FB72068F149D22AB30B94EC75CD56A10
:102F4800E378F1870E951CA32AB138CF46DD54EB00
:102F580062F97008811A932CA53EB740C952DB6408
:102F6800ED76FF89009B12AD24BF36C148D35AE5E0
:102F78006CF77E0A8318912EA73CB542CB50D966D0
:102F8800EF74FD8B029910AF26BD34C34AD158E7C0
:102F98006EF57C0C851E9728A13AB344CD56DF60A8
:102FA800E972FB8D049F16A920BB32C54CD75EE1A0
:102FB80068F37A0E871C952AA338B146CF54DD6290
:102FC800EB70F98F069D14AB22B930C74ED55CE380
:102FD8006AF17800112332465765748C9DAFBECADA
:102FE800DBE9F810013322564775649C8DBFAEDAD1
:102FF800CBF9E82130021367764455ADBC8E9FEBC0
:10300800FAC8D93120120377665445BDAC9E8FFBB0
:10301800EAD8C94253617004152736CEDFEDFC8823
:1030280099ABBA5243716014053726DECFFDEC9890
:1030380089BBAA6372405125340617EFFECCDDA97F
:10304800B88A9B7362504135241607FFEEDCCDB970
:10305800A89A8B8495A7B6C2D3E1F008192B3A4EEB
:103068005F6D7C9485B7A6D2C3F1E018093B2A5E50
:103078004F7D6CA5B48697E3F2C0D129380A1B6F3F
:103088007E4C5DB5A49687F3E2D0C139281A0B7F30
:103098006E5C4DC6D7E5F48091A3B24A5B69780CA3
:1030A8001D2F3ED6C7F5E49081B3A25A4B79681C10
:1030B8000D3F2EE7F6C4D5A1B082936B7A48592DFF
:1030C8003C0E1FF7E6D4C5B1A092837B6A58493DF0
:0330D8002C1E0F9C
:030023000245EBA8
:0B45EB00C0E0C083C082C0D075D018B3
:1045F600309870C298751301AD99203015BD550BD2
:10460600906177E4F0D230D2918058906F40EDF00F
:104616008051906F3DE07046906177E0FE2442F550
:1046260082E4346FF583EDF0EEB40106ED0490619B
:104636006FF0906177E0FF601190616FE0FEB51F4B
:104646001504906F3DF0C291800CED64556007C271
:1046560030906F40EDF0906177E004F08005906F48
:1046660040EDF030992F30312AD290906176E0FFFC
:104676009061B0E0FEB51F08C231D232C2908013FD
:1046860074422EF582E43470F583E0F5999061B0BA
:05469600E004F0C299F0
:09469B00D0D0D082D083D0E032EF
:103F5700C231C232C230E4906F3FF09061B0F0904E
:103F67006176F0F5109061B1F0906177F0F51390FC
:103F77007B79F0906852F0E4906104F0906104E07E
:103F8700FFC394085023906852E075F075A424622B
:103F9700F582E5F03468F58375F00DEF12252BE413
:103FA700F0906104E004F080D3906852E0FF75F070
:103FB70075A42455F582E5F03468F583E4F0EF75D0
:103FC700F00DA42406F582E43461F583E4F09061F2
:103FD70075F0906175E0FFC394085023906852E034
:103FE70075F068A42443F582E5F03471F58375F024
:103FF7000DEF12252BE4F0906175E004F080D3906B
:104007006852E004F0E064086003023F7EE49074C5
:1040170083F0906000F0906105F0906170F090611E
:10402700ADF0907142F0906175F0906104F0906886
:1040370052F09061ACF0C2ADF5C9D2CDD2CCC2C9B5
:10404700C2CAF5CDF5CC9061AEE0F5CBA3E0F5CAD9
:1040570085CBCD85CACCD29ED29CD2CAC2ACC298DF
:0B406700C29975B85075B750D2AC225A
:103E39008F2B303312907B33E0B4420B907B36E00A
:103E490064027003023F56907B34E054E324BE6061
:103E59003814603524E3605C147003023F1D24E1CB
:103E6900602724606003023F56907B3363A2019070
:103E79007B35E075F00DA42406F582E43461F58301
:103E890063A201AF2B1231B622907B3363A201905A
:103E99006170E075F00DA424FDF582E5F0346BF551
:103EA9008363A201906170E004F0E0543FF0AF2B0E
:103EB9001231B622907B35E075F075A42462F58243
:103EC900E5F03468F583C083C082907B36E0543FC7
:103ED900FF1313543FD082D08375F00D12252B7D2B
:103EE90033AF2B1231A4907B35E075F068A42443DD
:103EF900F582E5F03471F583C083C082907B36E0AA
:103F0900543FFF1313543FD082D08375F00D12250F
:103F19002BE4F022907B3363A201907B35E075F0AE
:103F290068A42443F582E5F03471F583C083C08227
:103F3900907B36E0543FFF1313543FD082D08375F2
:0E3F4900F00D12252B63A201AF2B1231B62210
:10193C00E4F52A906F3EE0FFE52AC39F4003021CAA
:10194C0036906105E0FF906170E06F606775F00D97
:10195C00EFA42401F582E5F0346CF583E02405F561
:10196C002BC3940E5033906105E075F00DA424FD4B
:10197C00F582E5F0346BF58363A2019061ACE02451
:10198C0003F582E43460F58363A201AF2B1231B608
:10199C009061ACE0252BF0800E30220B7E2E7F88E0
:1019AC00E4FBFDFC124072906105E004F0E0543F52
:1019BC00F0021C31906852E0FF75F075A42462F5BA
:1019CC0082E5F03468F583C083C082906104E0FE48
:1019DC00D082D08375F00D12252BE07003021AB55E
:1019EC0075F075EFA42466F582E5F03468F583751F
:1019FC00F00DEE12252BE02405F52BC3940E50456B
:101A0C00906852E075F075A42462F582E5F03468B4
:101A1C00F583C083C082906104E0D082D08375F0DE
:101A2C000D12252B63A2019061ACE02403F582E436
:101A3C003460F58363A201AF2B1231B69061ACE038
:101A4C00252BF0800E30220B7E2E7F88E4FBFDFCD4
:101A5C00124072906852E0FF75F075A42462F58212
:101A6C00E5F03468F583C083C082906104E0D082D5
:101A7C00D08375F00D12252BE4F0906104E004F096
:101A8C00E0C394085003021C31E4F075F075EFA428
:101A9C002455F582E5F03468F583E4F0906852E063
:101AAC0004F0E05407F0021C319061ADE0FF75F0DA
:101ABC000DA42406F582E43461F583E06078EF75BB
:101ACC00F00DA4240AF582E43461F583E02405F5D5
:101ADC002BC3940E50329061ADE075F00DA424062A
:101AEC00F582E43461F58363A2019061ACE02403D8
:101AFC00F582E43460F58363A201AF2B1231B6900A
:101B0C0061ACE0252BF0800E30220B7E2E7F88E41A
:101B1C00FBFDFC1240729061ADE075F00DA4240643
:101B2C00F582E43461F583E4F09061ADE004F0E01B
:101B3C005407F0021C319061ADE004F0E05407F062
:101B4C00907142E0FF75F068A42443F582E5F0340F
:101B5C0071F583C083C082906175E0FED082D08322
:101B6C0075F00D12252BE07003021C1975F068EF4F
:101B7C00A42447F582E5F03471F58375F00DEE126F
:101B8C00252BE02405F52BC3940E5045907142E0B3
:101B9C0075F068A42443F582E5F03471F583C083B5
:101BAC00C082906175E0D082D08375F00D12252B28
:101BBC0063A2019061ACE02403F582E43460F58308
:101BCC0063A201AF2B1231B69061ACE0252BF080F3
:101BDC000E30220B7E2E7F88E4FBFDFC12407290AF
:101BEC007142E075F068A42443F582E5F03471F598
:101BFC0083C083C082906175E0D082D08375F00D74
:101C0C0012252BE4F0906175E004F080189061755A
:101C1C00E004F0E0C39408400CE4F0907142E0045E
:101C2C00F0E05407F0052A02193F9061ACE0F52B67
:101C3C00E4F09070427455F0A3F0E52B2405A3F06A
:101C4C00E4A3F0906853E0907046F0906854E090F4
:101C5C007047F0E52B601190600363A2019070480F
:101C6C0063A201AF2B1231B6E4F56FF570E52B24AE
:101C7C0003F57290704563A201902EDB63A201AF55
:101C8C0072AE71AD70AC6F1231F28F728E718D704D
:101C9C008C6F7448252BF582E43470F583E570F075
:101CAC007449252BF582E43470F583E56FF0E52B50
:101CBC002408906176F0D231E49061B0F0906174B8
:101CCC00F0C2992099FDD2993022107E2E7F937C00
:0B1CDC00707D42906176E0FB124072C8
:011CE70022DA
:1026A600200B03C2AC22D2AC9061ADE075F00DA454
:1026B6002406F582E43461F583E0700A9061ADE0AA
:1026C60004F0E05407F0906852E0FF75F075A4241A
:1026D60062F582E5F03468F583C083C082906104B8
:1026E600E0D082D08375F00D12252BE07029906121
:1026F60004E004F0E0C39408401DE4F075F075EFC3
:10270600A42455F582E5F03468F583E4F090685228
:10271600E004F0E05407F0301620C216906F41E056
:10272600601204F0E0D394F0400A9080007480F0C8
:10273600C2AF80FE906174E004F030D844C2D890F5
:1027460061B1E0FF906F3FE0FDC39F5034E5742513
:10275600EAF5EA30D709E57325FA04F5FA8006E5C5
:102766007325FAF5FA74B22DF582E43461F583E047
:10277600FF906853E0B5070312193C906F3FE004E1
:10278600F030310F906174E0D39414400BC231D213
:10279600328005E4906174F0906F40E060127E2E06
:1027A6007F9F7C6F7D407B01124072E4906F40F00A
:1027B600906F3DE0FF7003022964F529E4F56FF59B
:1027C60070E52924FEF572906F4463A201902EDB1A
:1027D60063A201AF72AE71AD70AC6F1231F28F723F
:1027E6008E718D708C6FC230E4906F3DF0E5704550
:1027F6006F60262022030229647E2E7FA17C6F7DD6
:1028060042AB291240727F321252BE7E2E7F9F7CCF
:10281600007D6F7B021240722230220D7E2E7FAC2D
:102826007C6F7D42AB29124072906F44E0FB6401DD
:1028360060030228F5906F46E09061ABF06007E018
:1028460020E7030229649061ABE0547FF09068545E
:10285600F0E5E9240AF5EA30D707E5F904F5FA8048
:102866000385F9FAC2D8907CEDE014601B14602C45
:1028760024027035906F45E0FF7E007C067D1812BD
:1028860023EF8E738F748021906F45E0FF7E007C6E
:10289600017D861223EF8E738F74800D906F45E055
:1028A60075F0BEA485F073F574906F47E0FE541F73
:1028B6009061B1F0EEC413540704906F3EF0E4A3A8
:1028C600F0F5299061B1E0FFE529C39F4003022995
:1028D6006474482529F582E4346FF583E0FF74B209
:1028E6002529F582E43461F583EFF0052980D4903B
:1028F6006F45E0FF906853E06F7063EB24FC603235
:1029060014603E2402704930220B7E2E7FB6E4FB13
:10291600FDFC124072907B79E07043907B79740DD8
:10292600F0906F4763A201907B2363A201FF1231EF
:10293600B6223022297E2E7FC9E4FBFDFC124072AE
:102946002230221A7E2E7FCFE4FBFDFC124072223B
:0E29560030220B7E2E7FD6E4FBFDFC12407279
:012964002250
:100EE2000AC1EBEEEAE020D2C8D220EDE5F220E220
:100EF20020EAEEEDF4E8E3F3F0E0F6E8E820EFEEC6
:100F020020C0D4C12020000ACEF2E4E0FE20EFE0AF
:100F1200EAE5F220D2C8D22020000AC1EBEEEAE8CC
:100F2200F0F3FE20EFE0EAE5F220D2D120F120EF4B
:100F3200F0E8E7EDE0EAEEEC20EEF8E8E1EAE8219D
:100F420020000A53656E643A20000A526563204FFE
:100F52004B21000A435243206572726F7221000ACC
:100F6200CFE0EAE5F220EEF220F1E5F0E2E5F0E092
:100F7200212020000ACFE0EAE5F220D2D32020008F
:100F82000AC1EBEEEAE8F0EEE2EAE020D2D320205A
:100F9200003E2A2C312CCFE0F0E0ECE5F2F0FB2011
:100FA200F1E8EDF5F0EEEDEDEEE3EE20EFEEF0F22E
:100FB200E00A003E4C2C4230312C256C752CD1EAD3
:100FC200EEF0EEF1F2FC20EEE1ECE5EDE02C363055
:100FD200302C313230302C323430300A003E422C48
:100FE2004731302C2562752CC8EDE2E5F0F1E8FFBF
:100FF20020EDE020EFF0E8B8ECE50A003E422C4795
:1010020031312C2562752CC8EDE2E5F0F1E8FF20C4
:10101200EDE020EFE5F0E5E4E0F7E50A003E2A2CFA
:10102200312CCAEEEDF4E8E3F3F0E0F6E8FF20CA73
:10103200CF20C3D0C0CDC8D2202020312DE1EBEE8D
:10104200EA20D2D12C20322DE1EBEEEA20D2C8D216
:101052002C20332DE1EBEEEA20D2D32C20302DEFE1
:10106200F3F1F2EE200A003E532C4732302C257366
:101072002CF0E0E7ECE5F9E5EDE8E520E1EBEEEA5E
:10108200EEE220E220EAE0F0EAE0F1E53A0A003E90
:10109200422C4732322C2562752CD0E5E2E5F0F184
:1010A20020D2D10A003E422C4732332C2562752CC5
:1010B200C3F0F3EFEFFB20D2C8D220EDF3ECE5F062
:1010C200F3FEF2F1FF20F120F7B8F2EDEEE3EE0AC3
:1010D200003E422C4732342C2562752CD0E0F1F8C8
:1010E200E8F0E5EDEDFBE920EFF0EEF2EEEAEEEBF3
:1010F2000A003E2A2C312CCFF0EEF2EEEAEEEB2083
:10110200C8F1E5F2FC2DCCE0E3E8F1F2F0E0EBFC13
:10111200EDFBE920EDE020E0F1E8EDF5F0EEEDED9C
:10112200EEEC20EFEEF0F2F30A003E422C6B31348B
:101132002C2562752CC0EAF2E8E2E8F0EEE2E0F279
:10114200FC20EFEEF0F20A003E4C2C6B30352C25E1
:101152006C752CD1EAEEF0EEF1F2FC20EEE1ECE55A
:10116200EDE020EDE020EFEEF0F2F32C3130302C08
:101172003230302C3330302C3630302C313230306B
:101182002C323430302C343830302C393630302C4C
:1011920031393230302C33383430302C3537363028
:1011A200302C3131353230300A003E532C6B303620
:1011B2002C2562752CC0E4F0E5F120CACF20E4EBC7
:1011C200FF20ECE0E3E8F1F2F0E0EBE80A003E5346
:1011D2002C6B31322C2562752CCAEEEB2DE2EE20FF
:1011E200E1EBEEEAEEE220E220EEF2E2E5F2E520C9
:1011F20028EFE0EAE5F23D352B6E2A313320E1E0BB
:10120200E9F2290A003E532C6B31332C2562752CEE
:10121200C7E0E4E5F0E6EAE020F1F2E0F0F2E020F7
:10122200EFE5F0E5E4E0F7E828ECF1290A003E42B8
:101232002C6B30392C2562752CCDE520EFE5F0E5DD
:10124200E4E0E2E0F2FC20E4E8E0E3EDEEF1F2E8D3
:10125200EAF30A003E422C6B31302C2562752CCF0A
:10126200E5F0E5E7E0E3F0F3E7EAE020EFF0E8207D
:10127200EEF2F1F3F2F1F2E2E8E820EEE1ECE5ED74
:10128200E0203220ECE8ED2E0A003C4230313D00F5
:101292003C4731303D003C4731313D003C47323024
:1012A2003D003C4731323D003C4731343D003C4734
:1012B20032323D003C4732333D003C4732343D0040
:1012C2003C6B30353D003C6B30363D003C6B31337E
:1012D2003D003C6B30393D003C6B31303D003C6B96
:1012E20031343D000008040C020A060E0109050D06
:1012F200030B070F00112332465765748C9DAFBE56
:10130200CADBE9F810013322564775649C8DBFAEE3
:10131200DACBF9E82130021367764455ADBC8E9FD3
:10132200EBFAC8D93120120377665445BDAC9E8FC3
:10133200FBEAD8C94253617004152736CEDFEDFCB3
:101342008899ABBA5243716014053726DECFFDECA3
:101352009889BBAA6372405125340617EFFECCDD93
:10136200A9B88A9B7362504135241607FFEEDCCD83
:10137200B9A89A8B8495A7B6C2D3E1F008192B3A83
:101382004E5F6D7C9485B7A6D2C3F1E018093B2A63
:101392005E4F7D6CA5B48697E3F2C0D129380A1B53
:1013A2006F7E4C5DB5A49687F3E2D0C139281A0B43
:1013B2007F6E5C4DC6D7E5F48091A3B24A5B697833
:1013C2000C1D2F3ED6C7F5E49081B3A25A4B796823
:1013D2001C0D3F2EE7F6C4D5A1B082936B7A485913
:1013E2002D3C0E1FF7E6D4C5B1A092837B6A584903
:1013F2003D2C1E0F0089129B24AD36BF48C15AD323
:101402006CE57EF78108931AA52CB73EC940DB52E2
:10141200ED64FF76028B109926AF34BD4AC358D1D2
:101422006EE77CF5830A9118A72EB53CCB42D950C2
:10143200EF66FD74048D169F20A932BB4CC55ED7A2
:1014420068E17AF3850C971EA128B33ACD44DF56A2
:10145200E960FB72068F149D22AB30B94EC75CD592
:101462006AE378F1870E951CA32AB138CF46DD5482
:10147200EB62F97008811A932CA53EB740C952DB82
:1014820064ED76FF89009B12AD24BF36C148D35A62
:10149200E56CF77E0A8318912EA73CB542CB50D952
:1014A20066EF74FD8B029910AF26BD34C34AD15842
:1014B200E76EF57C0C851E9728A13AB344CD56DF22
:1014C20060E972FB8D049F16A920BB32C54CD75E22
:1014D200E168F37A0E871C952AA338B146CF54DD12
:1014E20062EB70F98F069D14AB22B930C74ED55C02
:0414F200E36AF17840
:104E2E00527B110000000000000000000000000096
:104E3E00000000000060207B7A20312020203520E9
:104E4E00202039202020313000000000000000001A
:104E5E00000000000000000000517B680080402030
:104E6E0010080402010000000000000000517B4603
:104E7E000000000000000000008040201008040226
:014E8E000122
:1051DD00907CE6E06FFC9013F693FE907CE5E06E1C
:0D51ED00A3F0AF04EF9012F693907CE5F074
:0151FA002292
:0100210022BC
:10529A00EF540F9012E693FEC454F0FEEFC4540F7D
:0452AA00932EFF221E
:024E90008D2E65
:104E9200AA06A9077531018A328933E4F52F125225
:104EA2006C8F30E530643C602AAB31AA32A933E51D
:104EB200301223DD74012533F533E43532F5320542
:104EC2002F12526C8F30E530643C6007E52FC3959A
:104ED2002E40D6E52FB52E0C74FF2533F53374FF23
:0E4EE2003532F532AB31AA32A933E41223DDAA
:014EF000229F
:101CE80020150302207EC21530192EE49078F9F0F1
:101CF800907CE3E024FEF5299078FAF0907AFEE0F3
:101D08009078FBF0A37408F0907BE163A2019078CF
:101D1800FD63A201AF291231B6907BE1E0907CEC23
:101D2800F0907BE2E0FE54F064F0707A907BE5E09E
:101D3800FD54F0FFC4540F2457F582E4347BF58337
:101D4800E0F52970037F0122907BE3E0FC640270D8
:101D58003FA3E064917039E52930E731907B337413
:101D680048F0A37461F0EE540F2457F582E4347BF5
:101D7800F583E0540F907B35F0907B377408F0EDD5
:101D8800540F75F008A4907B36F07F01227F012262
:101D9800EC6406600302207B907BE4E064916003BE
:101DA80002207B02207B907BE2E0540FFF2457F552
:101DB80082E4347BF583E07018907B42EFF03023A7
:101DC8000D7E0E7FE27C7B7D427B011240727F019B
:101DD80022907BE2E0540F2457F582E4347BF583AC
:101DE800E0FF20E703021F48907B337448F0A37498
:101DF80061F0EF540FA3F0907B377408F0300414AF
:101E0800907BE3E020E0047F0080027F10907B3627
:101E1800EFF08012907BE3E020E0047F1080027FE7
:101E280000907B36EFF0E4F529752A03E529C39481
:101E3800044003021F48907B36E04480F074E1259B
:101E48002AF582E4347BF583E0D394FA40067E13C6
:101E58007F888016AF2A052A74E12FF582E4347B47
:101E6800F583E075F014A4FFAEF0AD07AC06907BE7
:101E780038EFF0A3ECF074E1252AF582E4347BF521
:101E880083E0D394FA40067E137F888016AF2A0534
:101E98002A74E12FF582E4347BF583E075F014A40D
:101EA800FFAEF0AC06AD07907B3AEFF0A3ECF07410
:101EB800E1252AF582E4347BF583E0D394FA4006E1
:101EC8007E137F888016AF2A052A74E12FF582E4F5
:101ED800347BF583E075F014A4FFAEF0AC06AD07D3
:101EE800907B3CEFF0A3ECF074E1252AF582E43412
:101EF8007BF583E0D394FA40067E137F888016AF83
:101F08002A052A74E12FF582E4347BF583E075F025
:101F180014A4FFAEF0AC06907B3EEFF0A3ECF07F8C
:101F28000D123E3930230D7E0F7F097C7B7D367B79
:101F3800011240720529907B36E02404F0021E3419
:101F4800907BE2E0540F2457F582E4347BF583E07C
:101F580020E50302207B907BE3E030E71130230B80
:101F68007E0F7F1CE4FBFDFC1240727F0122907BF8
:101F7800337444F0A37420F0907BE2E0540F2457AC
:101F8800F582E4347BF583E0540F907B35F0E4A3CD
:101F9800F0A37406F0E4907B3CF0A3F0A3F0A3F068
:101FA800F529752A03E529C39402400302207B30F2
:101FB8001115AF2A052A74E12FF582E4347BF583E5
:101FC800E0FF12529A8010AF2A052A74E12FF58299
:101FD800E4347BF583E0FF907B38EFF0301115AFE8
:101FE8002A052A74E12FF582E4347BF583E0FF1299
:101FF800529A8010AF2A052A74E12FF582E4347BC7
:10200800F583E0FF907B39EFF0301115AF2A052AF0
:1020180074E12FF582E4347BF583E0FF12529A8055
:1020280010AF2A052A74E12FF582E4347BF583E0AA
:10203800FF907B3AEFF0301115AF2A052A74E12F93
:10204800F582E4347BF583E0FF12529A8010AF2AC0
:10205800052A74E12FF582E4347BF583E0FF907B59
:102068003BEFF07F0D123E390529907B35E004F0F7
:08207800021FAD7F01227F0071
:01208000223D
:104DBD00C226E4FE907CE2E064056044BF7E0BD227
:104DCD0005E4907B9CF0907CE2F0EF30E70B4375AF
:104DDD0001907CE2E004F080085375FEE4907CE2E3
:104DED00F0907B9CE004F0E0B4080D907CE8E57554
:104DFD00F0D226E4907B9CF0E57525E0F575800EEC
:104E0D00EF30E705D205A22622E4907CE2F0EF25F3
:0A4E1D00E0FF0EEE6408709CA22670
:014E27002268
:02480900AC07FA
:10480B00E4FE907B67E0FD25E0F0EC30E748E04408
:10481B0001F0202646907B45E004F0E06405703BF8
:10482B00F0907C61E004F0E0B40821907B67E0FF3E
:10483B000579E579AA787002057814F5828A83EFF9
:10484B00F0907CE4E004F0E4907C61F0907B67E016
:10485B00FF25E0F08005E4907B45F0907C61E0045F
:10486B00F0E0B40821907B67E0FF0579E579AA7841
:10487B007002057814F5828A83EFF0907CE4E004F3
:10488B00F0E4907C61F0EC25E0FC0EEE6408600334
:03489B0002480DC3
:01489E0022F7
:1052350075657E7562A0C208D20FC215D234C2133D
:0C524500C201C214D200C2121250AB22EF
:103BD400907CEE74FFF0A374B8F0E4907CEDF09068
:103BE4007CECF0907CE7F0907CEBF0907CE9741E28
:103BF400F0122C1BE4F52DF52CF52BF529752A0173
:103C0400747A2529F582E4347BF583E0FF7003029E
:103C14003CEEE52AC394104003023CEEEFB42004CA
:103C2400052980DC747A2529F9E4347BFA7B01C008
:103C3400031B8B31753200753300E4F534D0031265
:103C440032C41225373C65000000003C85000000AA
:103C5400013CA0000000023CB90000000300003C4D
:103C6400D0AF2A052A74572FF582E4347BF583E418
:103C7400F0E52B6004052B052BE52C604F052C800B
:103C84004BE52B4420FFAE2A052A74572EF582E417
:103C9400347BF583EFF0052B052B8030E52C448035
:103CA400FFAE2A052A74572EF582E4347BF583EFA0
:103CB400F0052C8017E52D4440FFAE2A052A7457E1
:103CC4002EF582E4347BF583EFF0052D747A2529F3
:103CD400F582E4347BF583E0FF64207003023C0446
:103CE400EF7003023C04052980E2E52AC3941050D6
:103CF40012AF2A052A74572FF582E4347BF583E446
:0F3D0400F080E7123F57124EF12019031252358B
:013D1300228D
:023D1400AB05FD
:103D1600907CE5E0907D02F0907CE6E0907D03F0FB
:103D2600E4907CE4F0907B45F0907CE5F0A3F08E87
:103D36002A8F2B75787C7579623010288579828573
:103D460078837405F00579E57970020578F5828542
:103D560078837455F00579E57970020578907CE4EE
:103D6600E02402F0857982857883747EF00579E512
:103D76007970020578907CE4E004F0E4907C61F0D0
:103D8600907D00F0907D00E0C39B504E852B828590
:103D96002A83E0FF12529A907D01EFF0907CE6E0D4
:103DA6006F907D01F0E0FF9013F693FE907CE5E0C6
:103DB6006EA3F0EF9012F693907CE5F0052BE52BC1
:103DC600AE2A7002052A14F5828E83E0FFC22612FF
:103DD6004809907D00E004F080AA907CE6E0FF129E
:103DE600529AC226124809907CE5E0FF12529AC206
:103DF60026124809D2267F7E124809D226E4FF12EF
:103E06004809D226E4FF124809D2017C7C7D628CE7
:103E1600788D7930230C7E0F7F44907CE4E0FB1292
:103E26004072907D02E0907CE5F0907D03E0907C0E
:023E3600E6F0B4
:013E38002267
:10525100907BE07402F0907CECE0907BA0F0A37472
:0B52610018F0D212907CE97464F02277
:1051BC008F2920011B30120CC2127E7B7FA0AD29DF
:1051CC00123D14227E777FFDE52924FCFD123D144F
:0151DC0022B0
:1046A400E4FF0F2489F582E43475F5837408F00F70
:1046B40074892401F582E43475F583E4F07C7B7D10
:1046C40016FEED1DAA0470011CF5828A83E0FBAA84
:1046D400070F74892AF582E43475F583EBF00EBE76
:1046E40004E07C7B7D1AE4FEED1DAA0470011CF538
:1046F400828A83E0FBAA070F74892AF582E4347561
:10470400F583EBF00EBE04E07C7B7D1EE4FEED1D24
:10471400AA0470011CF5828A83E0FBAA070F74893E
:104724002AF582E43475F583EBF00EBE04E07C7B5D
:104734007D22E4FEED1DAA0470011CF5828A83E04B
:10474400FBAA070F74892AF582E43475F583EBF02C
:044754000EBE04E0B1
:01475800223E
:1035EF00200803023720E5605438655B700302370B
:1035FF0073E55B24085438F55B131313541F244BE6
:10360F00F8E6907B9FF0200537200734E0FF124D3E
:10361F00BD50D3907CE8E0FF12529A1251DD907C9E
:10362F00E8E0857782857683F00577E57770020588
:10363F0076907CE3E004F0E0D3942040A9D20722F7
:10364F00907CE3E0FBD394024008907BE1E06002C2
:10365F00D215C208C205E4F549D234907CE6E0FFEA
:10366F00907CE5E04F703A30230B7E0F7F4C7C7BD4
:10367F007DE1124072907B13E0FCA3E0FDA3E0FE1E
:10368F00A3E0FFE4FAF9F8EF2401FFEA3EFEE93D7B
:10369F00FDE83CFC907B131224EEE4907CEAF08072
:1036AF006BC2153023107E0F7F557C7B7DE1907CA4
:1036BF00E3E0FB124072907B1BE0FCA3E0FDA3E074
:1036CF00FEA3E0FFE4FAF9F8EF2401FFEA3EFEE97A
:1036DF003DFDE83CFC907B1B1224EE20071FD20817
:1036EF00E4907CE3F0907CE2F0907CE6F0907CE557
:1036FF00F0907B9CF0C23475767B7577E1907CEA15
:10370F00E004F0D394054004D202E4F0C20702357E
:10371F00F5203450E54B647E702A300207F549D20C
:10372F0034C20222D200D208E4907CE3F0907CE213
:10373F00F0907CE6F0907CE5F0907B9CF075767BCA
:10374F007577E122E54BB4A016200613D200907BCB
:10375F0043E0FFA3E0907B9DCFF0A3EFF0C209E41D
:05376F00F549D23422EF
:1029650030180AC218907B9AE0600214F030162CD9
:10297500907CE9E0601814F07014907CECE060083D
:102985002012051252518006907CE9E004F0907CFB
:10299500EBE0600814F07004907B79F01226A690A5
:1029A5007B79E07003022A78907CEBE06003022AD1
:1029B5007830230D7E0F7F617C7B7D237B06124063
:1029C50072907BE0740AF0907CECE0907BA0F09034
:1029D5007B26E060047F1180027F12907BA1EFF0DF
:1029E500907B25E0FF131313541F04FE2468F58222
:1029F500E4347BF583E0907BA2F074462EF582E407
:102A0500347BF583E0907BA3F0EF54072469F582CE
:102A1500E4347BF583E0907BA4F0907BA1E0540F38
:102A2500FFBF0108907B69E0F4FF8006907B6AE0B8
:102A3500F4FF907BA5EFF0A374FFF0907BA2E0F488
:102A4500907BA7F0907BA3E0F4907BA8F0907BA40B
:102A5500E0F4907BA9F0D21230230D7E0F7F767CB7
:102A65007B7DA07B0A124072E4907B79F0907CEB31
:102A75007408F0907CEBE06015907B79E0600FE4E2
:102A8500F030230A7E0F7F82FBFDFC124072123567
:102A9500EF201903121CE8201303022B27E56165BB
:102AA5005C604EE56124085438FFE55C54386F607E
:102AB500047E0180027E00907CE4E060047D01805C
:102AC500027D00EE5D7003022C1A0579E579AC787C
:102AD5007002057814F5828C83E0FEE5611313130B
:102AE500541F2453F8A6068F61907CE4E014F0800F
:102AF500B2C213C201907B17E0FCA3E0FDA3E0FE88
:102B0500A3E0FFE4FAF9F8EF2401FFEA3EFEE93D10
:102B1500FDE83CFC907B171224EED214E4907B9ADE
:102B2500F022300803022C1A300137E561655C603C
:102B350003022C1A0579E579AE787002057814F54B
:102B4500828E83E0FFE561131313541F2453F8A607
:102B550007E56124085438F561907CE4E014F0D26F
:102B65001322301209907BE0E0FF1251BC22E5618F
:102B7500655C6003022C1A300303022C1A20002521
:102B8500907B1FE0FCA3E0FDA3E0FEA3E0FFE4FAD9
:102B9500F9F8EF2401FFEA3EFEE93DFDE83CFC9033
:102BA5007B1F1224EEC200E561131313541F245337
:102BB500F876AAE56124085438F561131313541FF8
:102BC5002453F876A0E56124085438F561131313EE
:102BD500541F2453F8E4F6E56124085438F56113CD
:102BE5001313541F2453F8E4F6E56124085438F50B
:102BF50061131313541F2453F8E4F6E561240854B4
:102C050038F561131313541F2453F8E4F6E56124D2
:052C1500085438F561D0
:012C1A002297
:0B002600301405C2147F01227F00226D
:103A63007BFF7A0F79931220E3907CEDE06033A320
:103A7300E0FEA3E0FFC3E49FFFE49EFEAB07FA333F
:103A830095E0F9F87F007EC27D017C0012243D8F12
:103A9300348E338D328C317BFF7A0F79B51220E36C
:103AA3008032907CEEE0FEA3E0FFC3E49FFFE49E40
:103AB300FEAB07FA3395E0F9F8E47F207E1CFDFCAA
:103AC30012243D8F348E338D328C317BFF7A0F7904
:103AD300B51220E37BFF7A0F79DFA20DE433F531D2
:103AE3001220E37BFF7A0F79FEA20CE433F5311247
:103AF30020E37BFF7A10791F1220E37531017532C1
:103B03007B75337A7BFF7A1079691220E37BFF7A26
:103B1300107991A211E433F5311220E37BFF7A107F
:103B230079A7A204E433F5311220E37BFF7A1079FD
:103B3300D3A20AE433F5311220E37BFF7A1079F440
:103B43001220E37BFF7A11792CA20BE433F53112B7
:103B530020E39061AEE0FEA3E0FFC3E49FFFE49E99
:103B6300FEAB07FA3395E0F9F87F007E8C7D0A7C83
:103B73000012243D8F348E338D328C317BFF7A11CA
:103B8300794A1220E37BFF7A1179AC906853E0F510
:103B9300311220E37BFF7A1179D0906F3EE0F5314B
:103BA3001220E37BFF7A127907906173E0F53112FB
:103BB30020E37BFF7A127930A233E433F53112200C
:103BC300E37BFF7A127956906F41E0F5311220E3DF
:013BD30022CF
:102C1B007E127F8C124AC9EF4E7003022CF1124FB9
:102C2B004F907D001224EEE4FFFEFDFC907D00E052
:102C3B00F8A3E0F9A3E0FAA3E0FBC31224DD7003D1
:102C4B00022D01907D00E0F8A3E0A3E0A3E07F005C
:102C5B007EC27D017C0012243D1224CF907CEEEECF
:102C6B00F0A3EFF0E47F607E09FDFC907D00E0F8BF
:102C7B00A3E0F9A3E0FAA3E0FBC31224DD700590F7
:102C8B007CED04F0E47FB07E04FDFC907D00E0F869
:102C9B00A3E0F9A3E0FAA3E0FBC31224DD700690D6
:102CAB007CED7402F0E47F587E02FDFC907D00E029
:102CBB00F8A3E0F9A3E0FAA3E0FBC31224DD70361E
:102CCB00907CEDF0907D00E0F8A3E0A3E0A3E0E4BE
:102CDB007F207E1CFDFC12243D1224CF907CEEEE57
:102CEB00F0A3EFF08010907CEE74FFF0A374D0F0A3
:102CFB00907CED7401F07E127F92124AC9EF4E6008
:102D0B000C12526CEF24D024FF920D8002C20D7E68
:102D1B00127F98124AC9EF4E600C12526CEF24D0FE
:102D2B0024FF920C8002C20C7E127F9E124AC9EFC6
:102D3B004E60097E7B7F7A7D20124E907E127FA49F
:102D4B00124AC9EF4E600C12526CEF24D024FF9242
:102D5B00038002C2037E127FAA124AC9EF4E600C97
:102D6B0012526CEF24D024FF92108002C2107E12FC
:102D7B007FB0124AC9EF4E600C12526CEF24D02474
:102D8B00FF92118002C2117E127FB6124AC9EF4E1A
:102D9B00600C12526CEF24D024FF92048002D204F8
:102DAB007E127FBC124AC9EF4E600C12526CEF249C
:102DBB00D024FF920A8002C20A7E127FC2124AC935
:102DCB00EF4E6023124F4FA804A905AA06AB077F4D
:102DDB00007E8C7D0A7C0012243D1224CF9061AEC4
:102DEB00EEF0A3EFF0800A9061AE74FFF0A374B81D
:102DFB00F07E127FC8124AC9EF4E600A124F4F90F5
:102E0B006853EFF080069068537401F0906F3E7436
:102E1B0001F07E127FCE124AC9EF4E600A124F4F5D
:102E2B00906173EFF08005E4906173F07E127FD4B4
:102E3B00124AC9EF4E600C12526CEF24D024FF9251
:102E4B00338002D2337E127FDA124AC9EF4E600C06
:102E5B0012526CEF24D0906F41F08005E4906F41DB
:102E6B00F07E127FE0124AC9EF4E600C12526CEFEB
:0C2E7B0024D024FF920B8002C20B7F00C9
:012E87002228
:03001E00C2AE224D
:0A52BE00E4FEEEC39F50030E80F8DB
:0152C80022C3
:1051FB00A2AF9226C2AF438E2075D2028F828E83CE
:0C520B00E0FFE4F5D2538EDFA22692AF44
:015217002274
:10515000E5D220E0FBA2AF9226C2AF43D2028F82FB
:105160008E83EDF075D25063D250A22692AFE5D275
:0351700020E0FB41
:015173002219
:104C5700E4FDED2401FFE433FE1251FB74BA2DF598
:104C670082E43477F583EFF00DBD3FE6E4FDED24F4
:104C77007FFFE433FE1251FB74B12DF582E43475E6
:104C8700F583EFF074B12DF582E43475F583E070A8
:104C97001B74B12DF582E43475F5837420F074B27A
:104CA7002DF582E43475F583E4F080040DBD80BEF4
:104CB700E4907630F0FDEDFF7E001251FB74312D4C
:0D4CC700F582E43476F583EFF00DBDFEE9D3
:014CD40022BD
:02511C008B2ED8
:10511E00A2AF9226C2AF85A22F53A2FE8E838F829C
:10512E0005A28C838D8274091232B2E52E53A2FE33
:10513E0043A2201232B453A2DF852FA2A22692AF31
:01514E00FF61
:01514F00223D
:10521800A2AF9226C2AF8C838D82EF1232B243A224
:0C522800201232B453A2DFA22692AFFF86
:015234002257
:025174008F2981
:10517600A2AF9226C2AFE4F5838D8274061232B2D4
:10518600E52943A2201232B453A2DFA22692AF7FB2
:015196000117
:0151970022F5
:025198008F295D
:10519A00A2AF9226C2AFE4F5838D82740A1232B2AC
:1051AA00E52943A2201232B453A2DFA22692AF7F8E
:0151BA0001F3
:0151BB0022D1
:1030DB00A907E7FFA805EF93C3966008403B74FC74
:1030EB002FFF80F00F08EF93C3966008402B74FB03
:1030FB002FFF80E00F08EF93C3966008401B74FA14
:10310B002FFF80D00F08EF93D3966008400B74F914
:10311B002FFF80C01F1F1F1F1FEF54FEF80303F765
:10312B00E893FC08E893FD08E893FE08E893FF2278
:10313B0009E993C39D6008402974FB29F980F109C3
:10314B00E993C39E6008401A74FA29F980E209E9F1
:10315B0093D39F6008400B74F929F980D31919197F
:10316B001919E9C313C313FF22740093F8ECC39826
:10317B004024701F740193F8EDC3984019701474B8
:0E318B000293F8EEC398400E7009740393F897
:10319900EFC39840037F00227F0122EDF8E6F00893
:1031A900A3DFFA22EDF8E0F608A3DFFA22E0A36331
:1031B900A201F0A363A201DFF475A2002263A201B8
:1031C900F0A363A20122E0A363A201F0A363A20119
:1031D900E0A363A201F0A363A201E463A201F0A347
:1031E90063A201DFE175A20022E0A363A2016DFEE3
:1031F900936CFDEE058393FC158363A201DFEA75E9
:10320900A200227F00E493A363A201F00F600CA344
:10321900E583C2E3F58363A20180EA75A20022E097
:10322900A363A201F0A3E583C2E3F58363A201DFEF
:10323900EE75A20022E0A363A201F0A3E583C2E434
:10324900D2E3F58363A201DFEC75A20022E0A36358
:10325900A201F0A3E58344F8C2E5F58363A201DF87
:10326900EC75A20022E583C2E3F583E0A363A20122
:10327900F0A363A201DFEE75A20022E583C2E4D2C6
:0A328900E3F583E0A363A201F0A3C4
:1032930063A201DFEC75A20022E58344F8F583E025
:1032A300A363A201F0A363A201DFEE75A20022F9DA
:1032B30022C002C004C00612FFF0D006D004D00220
:0132C30022E8
:0300000002492F83
:0C492F00787FE4F6D8FD758179024976A6
:1023DD00BB010689828A83F0225002F722BBFE01DF
:0223ED00F322D9
:1023EF00EF8DF0A4A8F0CF8CF0A428CE8DF0A42E02
:0223FF00FE22BC
:1024010075F008758200EF2FFFEE33FECD33CDCC92
:1024110033CCC58233C5829BED9AEC99E582984015
:102421000CF582EE9BFEED9AFDEC99FC0FD5F0D6F2
:10243100E4CEFBE4CDFAE4CCF9A88222B800C1B91C
:102441000059BA002DEC8BF084CFCECDFCE5F0CB5A
:10245100F97818EF2FFFEE33FEED33FDEC33FCEB93
:1024610033FB10D703994004EB99FB0FD8E5E4F94E
:10247100FA227818EF2FFFEE33FEED33FDEC33FC3B
:10248100C933C910D7059BE99A4007EC9BFCE99A2F
:10249100F90FD8E0E4C9FAE4CCFB2275F010EF2F74
:1024A100FFEE33FEED33FDCC33CCC833C810D70774
:1024B1009BEC9AE899400AED9BFDEC9AFCE899F8AF
:0E24C1000FD5F0DAE4CDFBE4CCFAE4C8F92242
:0E24CF00C3E49FFFE49EFEE49DFDE49CFC221E
:1024DD00EB9FF5F0EA9E42F0E99D42F0E89C45F055
:0124ED0022CC
:0C24EE00ECF0A3EDF0A3EEF0A3EFF02261
:1024FA00A8828583F0D083D0821225111225111269
:10250A002511122511E473E493A3C583C5F0C5838D
:10251A00C8C582C8F0A3C583C5F0C583C8C582C82B
:01252A00228E
:0C252B00A42582F582E5F03583F58322BB
:10253700D083D082E4937012740193700DA3A39398
:10254700F8740193F5828883E4737402936C7012B4
:102557007403936D700C7404936E70067405936F17
:0A25670060DDA3A3A3A3A3A380CA11
:10208100E53D2431F8E6053D22782E302D027831E8
:10209100E475F0011226060225712026EB7F2ED26F
:1020A100268018EF540F2490D43440D4FF302A0BEB
:1020B100EF24BFB41A0050032461FFE53E6002150E
:1020C1003E0541E54170020540302D0D782EE47545
:1020D100F001122606EF0223DD0250627403D22DB5
:1020E1008003E4C22DF53D8B2E8A2F8930E4F53E25
:1020F100F540F541E53E60077F201220BC80F57573
:102101003FFFC227C226C228C229C22BC22CC22E1F
:1021110012208AFF700D302D057F001220CDAF41B6
:10212100AE4022B4255FC2D5C22A12208AFF24D034
:10213100B40A00501A75F00A783E30D50508B6FF8A
:102141000106C6A426F620D5047002D22980D9241E
:10215100CFB41A00EF5004C2E5D22A0222CDD22711
:1021610080C6D22680C0D22880BCD2D580BAD22BDC
:1021710080B47F201220BC2028077401B53E0040A6
:10218100F1122081FF1220BC0220F5D22ED22C8028
:1021910095122081FB122081FA122081F94A4B709D
:1021A10006799E7A237BFF20282EE53E602A7E0059
:1021B1008E8275830012258A60060EEE653F70F0EF
:1021C100C2D5EBC0E0EAC0E0E9C0E0EE122314D0D2
:1021D100E0F9D0E0FAD0E0FB122571FF60AAEBC074
:1021E100E0EAC0E0E9C0E01220BCD0E02401F9D06F
:1021F100E03400FAD0E0FBE53F0460DCD53FD98054
:10220100877BFF7A237910D228809C79108002790C
:1022110008C22CC22E8008D2D5790A8004790AC25C
:10222100D5E53F047002F53FE4FAFDFEFF1220817F
:10223100FC7B08202713122081FD7B1030260A1217
:102241002081FE122081FF7B20EC3382D592D55074
:1022510013C3E43026069FFFE49EFEE42027039D7E
:10226100FDE49CFCE4CBF8C227EC700CCFCECDCCC6
:10227100E824F8F870F38017C3EF33FFEE33FEED77
:1022810033FDEC33FCEB33FB994002FB0FD8E9EB58
:10229100302705F8D0E0C448B227C0E00AEC4D4E23
:1022A1004F78207B0070C2EAB53F0040BCC0E0120D
:1022B1002316D0F0D0E0202704C4C0E0C4B227C068
:1022C100F01220A5D0F0D5F0EB0220F51226652101
:1022D1009253220C5821634C215F4222104F221845
:0F22E10044221849217843221E55220246220228
:1022F0004522024723BE5021672D216B2E218E2BB4
:10230000216F23218C2023A72A2127480000218622
:102310003F3F3F00790AA2D5202914302B09B9107C
:10232000020404B9080104A2D5202C0250010420A3
:1023300028689228B53E005034C0E07F203029192B
:102340007F30A228722C722B500F12236DC228C22C
:102350002CC22BC22E7F30800F302B03E9C0E0123D
:1023600020BC302B03D0E0F9D0E0B53ECC302B17A9
:102370007F30B9100C1220BC7F58302A077F78803C
:1023800003B908031220BC3028057F2D0220BC7F32
:1023900020202EF87F2B202CF322922880CF286E2D
:1023A000756C6C2900D2271220813027F8C227785B
:1023B0003E30D50108F60221272D504349581220FE
:1023C000812403B405004001E49023B9931220ADA9
:0D23D000743A1220ADD229753E0402220C91
:1032C4008B2E8A2F8930E4F53AF539F538F537F540
:1032D40035F536E532453345316012EBC0E0EAC0DE
:1032E400E0E9C0E0AB31AA32A933122616AB2E05B1
:1032F40030E530AA2F7002052F14F9122571F53B21
:10330400C394094007E53BD3940D40E1E53B6420B9
:1033140060DBE53BB42D054336038016E53BB42B57
:1033240005433601800C74FF2530F53074FF352FCA
:10333400F52FE53460046410703FAB2EAA2FA9303A
:1033440012257164306009E534702E75340A8029C1
:1033540090000112258AFF64786004EFB458134387
:10336400360175341074022530F530E4352FF52F0D
:103374008007E5347003753408AB2E0530E530AAB8
:103384002F7002052F14F9122571F53BC394614087
:103394000AE53BD3947A5003533BDF74D0253BF5C5
:1033A4003BC3940A400CE53B9411406D74F9253BF2
:1033B400F53BE53BD395345060433601853A3F8570
:1033C400393E85383D85373CAF347E00E4FCFDABA7
:1033D4003AAA39A938A8371225B7C8ECC8C9EDC923
:1033E400CAEECACBEFCBE4FCFDFEEB253BF53AEE8F
:1033F4003AF539ED39F538EC38F537AF3AAE39AD41
:1034040038FCAB3FAA3EA93DA83CD31224DD5003AF
:1034140002337D43360402337DE53620E003E48045
:103424002DE53245334531601EAB2EE53024FFF9DE
:10343400E52F34FFFAEBC0E0EAC0E0E9C0E0AB31CD
:10344400AA32A933122616E53630E20774FFFFFECE
:10345400FDFC22E536AF3AAE39AD38AC3730E10386
:043464000224CF224D
:10493B00020879E493A3F8E493A34003F68001F211
:10494B0008DFF48029E493A3F85407240CC8C3337D
:10495B00C4540F4420C8834004F456800146F6DF4C
:10496B00E4800B0102040810204080904E28E47E66
:10497B00019360BCA3FF543F30E509541FFEE49341
:10498B00A360010ECF54C025E060A840B8E493A308
:10499B00FAE493A3F8E493A3C8C582C8CAC583CA33
:1049AB00F0A3C8C582C8CAC583CADFE9DEE780BEEB
:014E8F000022
:10257100BB010689828A83E0225002E722BBFE0268
:09258100E32289828A83E493229B
:10258A00BB010CE58229F582E5833AF583E0225006
:10259A0006E92582F8E622BBFE06E92582F8E22250
:0D25AA00E58229F582E5833AF583E493226A
:1025B700E88FF0A4CC8BF0A42CFCE98EF0A42CFCC3
:1025C7008AF0EDA42CFCEA8EF0A4CDA8F08BF0A441
:1025D7002DCC3825F0FDE98FF0A42CCD35F0FCEBA0
:1025E7008EF0A4FEA9F0EB8FF0A4CFC5F02ECD3965
:0F25F700FEE43CFCEAA42DCE35F0FDE43CFC22D2
:10260600FAE6FB0808E6F925F0F618E6CA3AF622D5
:10261600BB011A89828A83D0F0D0E0F8D0E0F9D0E5
:10262600E0FAD0E0FBE8C0E0C0F00226945016E9DC
:10263600F8D083D082D0E0F9D0E0FAD0E0FBC082B7
:10264600C08302268BBBFE16E9F8D083D082D0E089
:0F265600F9D0E0FAD0E0FBC082C08302269D22BB
:10266500D083D082F8E4937012740193700DA3A304
:1026750093F8740193F5828883E473740293686018
:06268500EFA3A3A380DF18
:09268B00EBF608EAF608E9F62274
:09269400EBF0A3EAF0A3E9F02247
:09269D00EBF208EAF208E9F2226E
:00000001FF
